:020000020000FC
:0200000060C0DE
:020016003EC0EA
:10001A0000C04F935F930F935FB7409167004530DD
:10002A000CF403C0442740936700403041F493988E
:10003A0094989598929A00916600D6D070D04130E3
:10004A0041F4929894989598939A00916500CCD02F
:10005A0066D0423041F4929893989598949A009178
:10006A006400C2D05CD0433041F49298939894983B
:10007A00959A00916300B8D052D043954093670097
:10008A005FBF0F915F914F9118950F931F932F9315
:10009A003F930FB716B320916800122736B33093F7
:1000AA00680012FF03C000C0B29B01960FBF3F91C8
:1000BA002F911F910F9118950FED0DBF0EE701BB00
:1000CA0001EC07BB0CE108BB00E20BBF0CE100BD71
:1000DA0002E000BF05E003BF09E106BF01E009BF76
:1000EA0011241092670080E090E0789463D0969A89
:1000FA008AD0969888D0FACFEE24FF1841E1001FE3
:10010A00111F4A9509F40895EE1CFF1CE21AF30A1E
:10011A0020F4E20EF31E8894F2CF0894F0CF0F93E6
:10012A000FB800E40EB90BE10DB9769BFDCFC09A6A
:10013A00C0980F910895F89400E00CBD0CE30ABD35
:10014A0005E408BD03E00EBDB99A08B706FFFDCF66
:10015A00B99808B705FFFDCF0DD000E00CBD04E348
:10016A000ABD08B706FFFDCF00270EBD0FEF08BF77
:10017A0078940895B19B716008951F9313E308E082
:10018A001F9108950F93F894726000E00CBD01E08E
:10019A000ABD09E008BDB99A08B706FFFDCF90FC71
:1001AA00B99808B705FFFDCF00270EBD7D7F78946B
:1001BA000F910895F8945F9354E0A3E6B0E080931A
:1001CA0061009093620000916100109162002AE040
:1001DA0030E092DFED9200936100109362005A952D
:1001EA0091F75F91789408950F931F93ECE4F2E0EE
:1001FA001127E00FF11F04901F910F91089503EB4F
:10020A000A95F1F708950F931F932F9325E01FEF97
:10021A000FEF0A95F1F71A95D9F72A95C1F72F9199
:10022A001F910F9108950F931F930FEF1FEF1A95C8
:10023A00000000000000D9F70A95C1F71F910F913D
:0E024A000895C0F9A4B0999282F880909C00AB
:00000001FF
